:100000000C9461000C947E000C947E000C947E0095
:100010000C947E000C947E000C947E000C947E0068
:100020000C947E000C947E000C947E000C947E0058
:100030000C947E000C947E000C947E000C947E0048
:100040000C945F010C947E000C947E000C947E0056
:100050000C947E000C947E000C947E000C947E0028
:100060000C947E000C947E00000000002400270009
:100070002A0000000000250028002B0000000000DE
:1000800023002600290004040404040404040202DA
:100090000202020203030303030301020408102007
:1000A0004080010204081020010204081020000012
:1000B0000007000201000003040600000000000029
:1000C000000011241FBECFEFD4E0DEBFCDBF11E092
:1000D000A0E0B1E0E0E4F7E002C005900D92A030AE
:1000E000B107D9F711E0A0E0B1E001C01D92A9303D
:1000F000B107E1F70E9458010C949E030C94000094
:100100000F931F938C018DE061E00E942B028AE027
:1001100060E00E942B02212F332727FD3A958BE0C8
:100120006DE041E00E9478028DE061E00E942B02C8
:1001300010708BE06DE041E0202F0E9478028DE08E
:1001400061E00E942B028AE061E00E942B021F9175
:100150000F9108958F929F92AF92BF92CF92DF92AC
:10016000EF92FF920F931F934C01CB01BA0125E947
:100170003FEB46E552E40E9413030E94B9025B0183
:100180006C017B018C019EE015950795F794E7942F
:100190009A95D1F78FEF9FE3E822F922A822B9229E
:1001A000C4010E948000C50190640E948000C701C4
:1001B00090640E9480001F910F91FF90EF90DF905C
:1001C000CF90BF90AF909F908F900895CF93DF9383
:1001D000C1E0D0E088E090E240E050E06AE774E4FB
:1001E0000E94AA0068EE73E080E090E00E94A70100
:1001F0008AE090E240E050E06AE774E40E94AA00DE
:1002000068EE73E080E090E00E94A70188E290E24F
:1002100040E050E06AE774E40E94AA0068EE73E0F0
:1002200080E090E00E94A7012196C530D10591F6AB
:10023000C1E0D0E088E090E240E050E563EC77E494
:100240000E94AA0068EE73E080E090E00E94A7019F
:100250008AE090E240E050E563EC77E40E94AA0077
:1002600068EE73E080E090E00E94A70188E290E2EF
:1002700040E050E563EC77E40E94AA0068EE73E08A
:1002800080E090E00E94A7012196C530D10591F64B
:10029000DF91CF9108958AE061E00E940B028DE02A
:1002A00061E00E940B028BE061E00E940B02089566
:1002B0000E94D1010E944B010E94E600FDCF1F92D7
:1002C0000F920FB60F9211242F933F938F939F930A
:1002D000AF93BF938091040190910501A091060115
:1002E000B0910701309108010196A11DB11D232F86
:1002F0002D5F2D3720F02D570196A11DB11D2093A4
:1003000008018093040190930501A0930601B09326
:1003100007018091000190910101A0910201B0912B
:1003200003010196A11DB11D80930001909301016D
:10033000A0930201B0930301BF91AF919F918F9160
:100340003F912F910F900FBE0F901F901895EF9235
:10035000FF920F931F937B018C018FB7F89440910C
:1003600004015091050160910601709107018FBF52
:100370002FB7F8948091040190910501A091060196
:10038000B09107012FBF841B950BA60BB70BE81686
:10039000F9060A071B0760F71F910F91FF90EF9076
:1003A0000895789484B5826084BD84B5816084BDED
:1003B00085B5826085BD85B5816085BDEEE6F0E0DE
:1003C000808181608083E1E8F0E0808182608083C9
:1003D000808181608083E0E8F0E0808181608083BB
:1003E000E1EBF0E0808184608083E0EBF0E08081ED
:1003F00081608083EAE7F0E080818460808380818F
:100400008260808380818160808380818068808336
:100410001092C1000895282F30E0C90186569F4FE1
:10042000FC0194912A573F4FF9018491882391F060
:10043000E82FF0E0EE0FFF1FE859FF4FA591B491B0
:10044000662329F48C91909589238C9308958C913F
:10045000892B8C930895482F50E0CA0182559F4FF5
:10046000FC012491CA0186569F4FFC0194914A5782
:100470005F4FFA0134913323D1F1222331F123303C
:1004800021F4809180008F7705C0243031F4809171
:1004900080008F7D8093800018C0213019F484B5CE
:1004A0008F7704C0223021F484B58F7D84BD0DC0C8
:1004B000263021F48091B0008F7705C0273029F4D1
:1004C0008091B0008F7D8093B000E32FF0E0EE0FBD
:1004D000FF1FEE58FF4FA591B491662329F48C912C
:1004E000909589238C9308958C91892B8C930895F2
:1004F000BF92CF92DF92EF92FF920F931F93CF9311
:10050000DF93E82EF62EB42EC0E0D0E0022F10E0EC
:1005100087E0C82ED12CBB2041F4B8010C2E02C0BC
:10052000759567950A94E2F70AC0B6016C1B7D0BBE
:10053000C80102C0959587956A95E2F7BC01617084
:100540008E2D0E942B028F2D61E00E942B028F2D99
:1005500060E00E942B022196C830D105E1F6DF91C0
:10056000CF911F910F91FF90EF90DF90CF90BF90B0
:10057000089504D06894B11150C0089533D088F024
:100580009F5790F0B92F9927B751A0F0D1F0660F7F
:10059000771F881F991F1AF0BA95C9F712C0B1309A
:1005A00081F03AD0B1E0089537C0672F782F8827BF
:1005B000B85F39F0B93FCCF3869577956795B395D9
:1005C000D9F73EF490958095709561957F4F8F4F48
:1005D0009F4F089557FD9058440F551F59F05F3FA6
:1005E00071F04795880F97FB991F61F09F3F79F055
:1005F00087950895121613061406551FF2CF4695D7
:10060000F1DF08C0161617061806991FF1CF869558
:100610007105610508940895E894BB27662777273C
:10062000CB0197F908950BD078C069D028F06ED02F
:1006300018F0952309F05AC05FC01124EECFCADF2D
:10064000A0F3959FD1F3950F50E0551F629FF001E5
:10065000729FBB27F00DB11D639FAA27F00DB11D3E
:10066000AA1F649F6627B00DA11D661F829F2227C7
:10067000B00DA11D621F739FB00DA11D621F839F4E
:10068000A00D611D221F749F3327A00D611D231F24
:10069000849F600D211D822F762F6A2F11249F5772
:1006A00050408AF0E1F088234AF0EE0FFF1FBB1F95
:1006B000661F771F881F91505040A9F79E3F510534
:1006C00070F014C0AACF5F3FECF3983EDCF3869540
:1006D00077956795B795F795E7959F5FC1F7FE2BDF
:1006E000880F911D9695879597F9089597F99F67BB
:1006F00080E870E060E008959FEF80EC08950024AA
:100700000A941616170618060906089500240A9476
:1007100012161306140605060895092E0394000CFC
:1007200011F4882352F0BB0F40F4BF2B11F460FF8B
:1007300004C06F5F7F4F8F4F9F4F0895F894FFCF96
:00000001FF
